:020000040800F2
:10000000009000205D050008490500084B05000828
:1000100000000000000000000000000000000000E0
:100020000000000000000000000000004D05000876
:1000300000000000000000004F0500085105000806
:10004000AD050008AD050008AD050008AD050008C8
:10005000AD050008AD050008AD050008AD050008B8
:10006000AD050008AD050008AD050008AD050008A8
:10007000AD050008AD050008AD050008AD05000898
:10008000AD050008AD050008AD050008AD05000888
:10009000AD050008AD050008AD050008AD05000878
:1000A000AD050008AD050008AD050008AD05000868
:1000B000AD050008AD050008AD050008EE11AA5514
:1000C00010B5064C2378002B07D1054B002B02D02E
:1000D000044800E000BF0123237010BD3C04002051
:1000E0000000000058190008044B10B5002B03D085
:1000F0000349044800E000BF10BDC04600000000F6
:100100004004002058190008002243088B4274D391
:1001100003098B425FD3030A8B4244D3030B8B4208
:1001200028D3030C8B420DD3FF22090212BA030C11
:100130008B4202D31212090265D0030B8B4219D3F2
:1001400000E0090AC30B8B4201D3CB03C01A524112
:10015000830B8B4201D38B03C01A5241430B8B425A
:1001600001D34B03C01A5241030B8B4201D30B0343
:10017000C01A5241C30A8B4201D3CB02C01A52416A
:10018000830A8B4201D38B02C01A5241430A8B422D
:1001900001D34B02C01A5241030A8B4201D30B0216
:1001A000C01A5241CDD2C3098B4201D3CB01C01A30
:1001B000524183098B4201D38B01C01A524143093A
:1001C0008B4201D34B01C01A524103098B4201D328
:1001D0000B01C01A5241C3088B4201D3CB00C01A95
:1001E000524183088B4201D38B00C01A524143080D
:1001F0008B4201D34B00C01A5241411A00D2014632
:10020000524110467047FFE701B5002000F006F8A4
:1002100002BDC0460029F7D076E770477047C04658
:1002200010B500F0C7F800F095F800F031F810BDF7
:1002300010B500F097F800F089F810BD10B50A4825
:100240000A4B0360E1231B02436000238360C36009
:10025000036183610C224261C36180221201026248
:10026000436201F049FA10BD5804002000440040E8
:1002700010B5010000230122044801F05FF90028B5
:1002800001D0002010BD0120FCE7C046580400202A
:1002900010B5FFF7D3FF10BDBFF34F8F034B044AD8
:1002A000DA60BFF34F8FC046FDE7C04600ED00E0C7
:1002B0000400FA0510B5214B1B78002B16D12048FD
:1002C000FFF7D6FF012800D010BD1D4B1B78013B66
:1002D000DBB2802BF8D800F06EF81A4B1860174B81
:1002E00001221A70184B00221A70EDE7164B18788D
:1002F0000130134BC018FFF7BBFF012813D1124A7E
:1003000013780133DBB213700D4A12789342DBD1BC
:100310000A4A002111700A4A5278FF2AD4D1022BCE
:10032000D2D1FFF7B9FF00F046F8064B1B686433E3
:100330009842C9D9014B00221A70C5E76E0500200A
:10034000EC040020700500206F05002010B5FFF7B9
:10035000B1FF10BD10B5A02000222021C00500F083
:100360008DFA10BD10B500F026F804000F4B1B6885
:10037000C31AFA22520093420ED30D4B1B78002B66
:100380000BD10B4BF43AFF3A1A70A0202021C00584
:1003900000F074FA054B1C6010BD054B00221A706A
:1003A000A0202021C00500F069FAF3E778050020BD
:1003B00074050020704710B500F046F910BD00002C
:1003C000014A024B9A6070470000000800ED00E00F
:1003D00030B587B01422002101A801F0E7F90E4BD7
:1003E0005A6B012422435A635B6B23400093009BAA
:1003F000A025ED0500222021280000F03FFA20234F
:100400000193029400230393049301A9280000F0B0
:1004100079F907B030BDC0460010024030B599B040
:10042000342200210BA801F0C1F91022002107A8F5
:1004300001F0BCF91C220021684601F0B7F98020C8
:10044000800000F021FA02240B9480235B000E93BD
:1004500000250F95C03B10931294139430221492F0
:10046000159380239B021693C023DB0517930BA8DB
:1004700000F034FA07230793089409950A9502219E
:1004800007A800F0D9FC00940295684600F0B4FD7E
:1004900019B030BD10B5FFF793FF00F0B5F8FFF7C6
:1004A000BDFFFFF795FFFFF7BBFEFFF7C1FEFCE7BF
:1004B00000B583B00B4B196C012211431964196C00
:1004C0000A400092009ADA6B802149050A43DA63F8
:1004D000DB6B0B400193019BC020C00000F0BAF819
:1004E00003B000BD0010024010B588B00400142213
:1004F000002103A801F05AF92268114B9A4201D059
:1005000008B010BD0F4BD96B802080020143D96326
:10051000DA6B02400192019A596B0122114359632F
:100520005B6B13400293029B0C2303930A3B0493DF
:100530000792A02003A9C00500F0E4F8E0E7C04658
:1005400000440040001002407047FEE770477047CB
:1005500010B500F06DF810BD704700000D488546DD
:10056000002103E00C4B5B58435004310B480C4B0B
:1005700042189A42F6D30B4A02E000231360043279
:10058000094B9A42F9D3FFF7E7FF01F0EDF8FFF7C7
:1005900081FFFEE700900020F8190008000000200D
:1005A0003C0400203C04002084050020FEE70000FD
:1005B00010B50400114B1978002901D1012010BD9C
:1005C000FA208000FFF7A0FD01000D4B1868FFF72F
:1005D0009BFD00F07BF800280DD1032C01D90120F0
:1005E000EDE7013000222100404200F03FF8054BCA
:1005F0001C600020E3E70120E1E7C0460400002082
:10060000000000200800002010B5084A116880236F
:100610005B000B4313600020FFF7CAFF041E02D0EB
:100620000124200010BDFFF743FFFAE7002002403D
:10063000034B1B78034A11685B1813607047C04670
:10064000040000207C050020014B18687047C0465C
:100650007C050020034A136803490B4003431360E1
:100660007047C04600000140FFF9FFFF70B5002849
:1006700011DB8308134EC0339B009D590324204097
:10068000C000FF2214008440A54389010A40824033
:100690002A439A5170BD0F230340083B9B08063341
:1006A0009B00094A944663445C6803221040C000E2
:1006B000FC3215008540AC4389010A408240224348
:1006C0005A60E7E700E100E000ED00E00138802338
:1006D0005B0498420FD2094A50600948036A1B0222
:1006E0001B0AC02109060B430362002393600733F2
:1006F0001360002070470120FCE7C04610E000E0D6
:1007000000ED00E0F0B500235AE084685F000326A6
:10071000BE40B4432600CC68BC4034438460446887
:1007200094434A681609012232409A4022434260AB
:1007300056E0DC080834A400265805321A4092001E
:100740000F279740BE430F6997403A00324322502B
:100750005AE0032600E00026A64034003C43434E06
:100760001832920094513468EA432600AE434F6831
:10077000FF0201D52C4326003C4C2660646826000D
:1007800016404F68BF0201D52C432600374C6660E7
:100790008426A459260016404F68BF0301D52C4378
:1007A0002600324C8427E6518026A45922404E6808
:1007B000F60301D52A0022432C4D80242A5101330F
:1007C0000C682200DA404FD001229A4025001540E3
:1007D0001442F4D003244E683440013C012C94D9D7
:1007E00003224C682240032A09D0C2685E00032419
:1007F000B440A24314008A68B2402243C26003227C
:100800004C682240022A94D004685E00032217003C
:10081000B740BC434F683A40B24022430260C02216
:1008200092024C681442CAD09A0814001834A400EA
:100830000E4EA75903241C40E4000F26A640B743E0
:10084000A026F605B04286D0094EB04208D0094E27
:10085000B04207D0084EB04200D17AE705267BE7C8
:10086000012679E7022677E7F0BDC046001802406E
:100870000004005000080050000C0050002A01D075
:10088000816170478162FCE710B5104A1368104916
:100890000B400343136080239B00984201D000204B
:1008A00010BD0C4B1B685800C01840000A49FFF7E8
:1008B0002BFC0130054B5B695B0503D5002803D099
:1008C0000138F7E70020EBE70320E9E7007000407C
:1008D000FFF9FFFF0000002040420F0070B582B01A
:1008E000041E00D129E20368DB0739D5C14A9168AB
:1008F00038230B40D16803220A40102B26D0082B46
:1009000026D063688022520293427FD0A022D20276
:10091000934200D181E0B74B1A68B7490A401A6088
:100920001A68B6490A401A606368002B00D180E05B
:10093000FFF78AFE0500AF4B1B689B0310D4FFF73F
:1009400083FE401B6428F6D90320F7E1032AD6D1A1
:10095000A84B1B689B0303D56368002B00D1EFE114
:1009600023689B0731D5A34A936838210B40D1688F
:1009700003220A40102B6AD0002B6BD19D4A1268CB
:10098000520503D5E268002A00D1DBE199484268AC
:100990009B490A40616909020A434260002B0DD15C
:1009A000036898490B4021690B4303600368DB0A25
:1009B00007221A40944BD340944A1360944B186812
:1009C000FFF7F6FD002800D0BEE123681B0700D426
:1009D00081E0884B9A6838231340182B73D0A369A1
:1009E000002B00D1B4E0834A136E01210B43136640
:1009F000FFF72AFE05007F4B1B6E9B076BD4FFF7AA
:100A000023FE401B0228F6D9032097E1794A11689A
:100A100080235B020B43136086E7764B19688022C4
:100A2000D2020A431A601968802252020A431A60ED
:100A30007AE7FFF709FE05006E4B1B689B038FD515
:100A4000FFF702FE401B6428F6D9032076E1022A54
:100A500092D193E7E368002B22D0664A1368694974
:100A60000B4021690B431360116880235B000B432B
:100A70001360FFF7E9FD05005E4B1B685B0506D4BC
:100A8000FFF7E2FD401B0228F6D9032056E1594941
:100A90004B685B4A13406269120213434B6094E750
:100AA000544A13685B490B401360FFF7CDFD050006
:100AB000504B1B685B0588D5FFF7C6FD401B02281D
:100AC000F6D903203AE14B4B1B6E9B0703D5A36974
:100AD000002B00D13AE123685B0700D4A2E0454B2C
:100AE0009A6838231340202B45D0424BDB6BDB0048
:100AF0004AD4404AD16B802040050143D163D36B77
:100B000003400193019B0125434B1B68DB053DD549
:100B1000A368012B4ED0052B52D0364BDA6D012144
:100B20008A43DA65DA6D03318A43DA65A368002BFC
:100B300050D0FFF789FD06002E4BDB6D9B076FD46D
:100B4000FFF782FD801B354B9842F5D90320F5E075
:100B5000284A136E01218B431366FFF775FD0500CC
:100B6000244B1B6E9B07B6D5FFF76EFD401B02287A
:100B7000F6D90320E2E01F4BDB6D9B0752D5A3683B
:100B8000002B4FD10120D9E00025BDE7224A116892
:100B900080235B000B431360FFF756FD06001E4BDE
:100BA0001B68DB05B4D4FFF74FFD801B0228F6D984
:100BB0000320C3E00F4AD36D01210B43D365B5E792
:100BC0000C4BDA6D04210A43DA65DA6D03390A4306
:100BD000DA65ABE7FFF738FD0600064BDB6D9B07D8
:100BE0001ED5FFF731FD801B0C4B9842F5D9032031
:100BF000A4E0C04600100240FFFFFEFFFFFFFBFF26
:100C0000FF80FFFFFFC7FFFF0024F400000000206B
:100C100008000020FFFEFFFF007000408813000066
:100C2000012D1ED0E369002B00D191E04F4A91685D
:100C300038220A40102A5ED0022B18D04B4A136883
:100C40004B490B401360FFF7FFFC0400474B1B6848
:100C50009B0149D5FFF7F8FC001B0228F6D90320B9
:100C60006CE0424AD36B43490B40D363DAE73F4A17
:100C700013683F490B401360FFF7E6FC05003B4B50
:100C80001B689B0106D5FFF7DFFC401B0228F6D945
:100C9000032053E0354AD36837491940236A606A14
:100CA0000343A06A00020343E06A0343206B03434B
:100CB0000B43D360116880235B040B431360D1683E
:100CC00080235B050B43D360FFF7BEFC0400274B7A
:100CD0001B689B0106D4FFF7B7FC001B0228F6D95E
:100CE00003202BE0002029E0204AD36823490B4051
:100CF000D360002022E0012B2CD01C4BDA680323A8
:100D00001340216A8B4227D170231340616A8B42C2
:100D100024D1FE21C9011140A36A1B0299421FD1AF
:100D2000F8239B031340E16A8B421BD1520F5207F9
:100D3000236B9A4218D1002000E0012002B070BD60
:100D40000120FBE70120F9E70120F7E70120F5E7A3
:100D50000020F3E70120F1E70120EFE70120EDE7B4
:100D60000120EBE70120E9E70120E7E7001002405E
:100D7000FFFFFFFEFFFFFFEF8C80C11FFCFFFEEFB8
:100D800010B52A4B9B6838221A4207D1274B1A68A4
:100D9000D20A072313402648D84010BD234B9A6837
:100DA00038231340082B3BD0204B9A68382313403C
:100DB000102B0DD01D4B9A6838231340202B31D0B7
:100DC0001A4B9A6838231340182B26D00020E4E7EA
:100DD000164AD1680D3B0B40D26812090721114019
:100DE0000131032B0FD01248FFF78EF90F4BDA6851
:100DF000120A7F23134058430C4BD968490F013125
:100E0000FFF782F9C9E70B48FFF77EF9074BDA686D
:100E1000120A7F2313405843EEE7FA20C001BCE7D3
:100E20000448BAE780200002B7E7C046001002403D
:100E30000024F40000127A0070B504000D000028B0
:100E400000D1AAE0574B1A68072313408B4221D3E5
:100E500023689A070ED55B0705D5534A9168E023AE
:100E6000DB010B439360504A936850490B40A168E3
:100E70000B4393602368DB0754D56368012B20D0B4
:100E8000022B3BD0002B3FD1474A126852051CD49D
:100E900001206AE0434A136807218B432B43136008
:100EA000FFF7D2FB06003F4B1A6807231340AB4203
:100EB000CED0FFF7C9FB801B3D4A9042F3D90320F7
:100EC00053E0394A1268920369D537498A68072086
:100ED000824313438B60FFF7B7FB0600324B9B68DE
:100EE00038221A406368DB009A421BD0FFF7ACFB44
:100EF000801B2F4B9842F1D9032036E02A4A126812
:100F00009201E2D4012030E0032B05D0264AD26DB5
:100F10009207DAD4012028E0234A126E9207D4D433
:100F2000012022E01F4B1A6807231340AB421DD853
:100F300023685B0706D51C4A93681E490B40E1688D
:100F40000B439360FFF71CFF174B9A68120A0F239D
:100F500013409B00184A9A581F231340D840174B40
:100F60001860174B1868FFF723FB70BD0D4A136814
:100F700007218B432B431360FFF766FB0600094BE9
:100F80001A6807231340AB42D2D0FFF75DFB801BEA
:100F9000074B9842F3D90320E7E70120E5E701205A
:100FA000E3E7C0460020024000100240FFF0FFFFD0
:100FB00088130000FF8FFFFF701900080000002059
:100FC00008000020014B18687047C0460000002050
:100FD00010B5FFF7F7FF064B9A68120B0723134073
:100FE0009B00044A9A581F231340D84010BDC046A6
:100FF00000100240B0190008F0B583B00400036887
:101000009B0362D5584BDB6BDB001ED4564AD16B79
:10101000802040050143D163D36B03400193019BC2
:101020000126524A116880235B000B431360FFF7CF
:101030000BFB05004D4B1B68DB0508D4FFF704FBD9
:10104000401B0228F6D9032502E00026E9E7002527
:10105000002D23D1444BD96DC02292000B001340C8
:10106000114210D0A2699A420DD03F4AD36D404937
:101070000B40D06D802149020143D165D16D3D48BF
:101080000140D165D365DB0710D4002D06D1364A67
:10109000D36D37490B40A1690B43D365012E15D1A0
:1010A000314AD36B34490B40D3630FE0FFF7CCFADE
:1010B00007002D4BDB6D9B07E7D4FFF7C5FAC01B7C
:1010C0002E4B9842F5D90325DFE700252368DB077F
:1010D00006D5254A536D03218B4361680B43536545
:1010E00023689B0706D5204A536D0C218B43A168CA
:1010F0000B43536523689B0606D51B4A536D204955
:101100000B40E1680B43536523685B040BD5164A1B
:10111000536D9B009B0861690B4353658023DB057E
:1011200062699A4211D023681B050BD50E4A536D94
:1011300014490B4021690B43536522698023DB016D
:101140009A4209D0280003B0F0BD074AD168802335
:101150005B020B43D360E6E7034AD16880235B025E
:101160000B43D360EEE7C046001002400070004021
:10117000FFFCFFFFFFFFFEFFFFFFFFEF88130000F4
:10118000FFCFFFFFFF3FFFFF10B504008368026938
:10119000134342691343C269134301680A686B48E9
:1011A000024013430B602268536869490B40E168B1
:1011B0000B435360226AA3691A4321688B68654810
:1011C000034013438B602268D36A0F218B43616A0B
:1011D0000B43D3622368604A93420AD05F4A93422A
:1011E0003ED05F4A93425CD05E4A934249D010237E
:1011F0000BE05D4B5A6D03231340022B43D02BD8D9
:10120000002B42D0012B42D10333E069802212022D
:10121000904248D0042B00D191E07AD8002B00D125
:1012200086E0022B73D15148636A5B00504A995A99
:10123000FEF76AFF63685B08C0186168FEF764FF29
:101240000200103A4B4B9A4200D97DE0236800041B
:10125000000CD860002062E0032B1AD10533D4E7DC
:10126000414B5A6D0C231340082B14D005D8002B8A
:1012700013D0042BC9D01023C7E70C2B0FD1043B8C
:10128000C3E70023C1E70223BFE70023BDE7102324
:10129000BBE71023B9E70223B7E70023B5E7102324
:1012A000B3E70023B1E7042B2ED023D8002B25D0A1
:1012B000022B1DD12D48636A5B002D4A995AFEF717
:1012C00023FF400063685B08C0186168FEF71CFFDD
:1012D0000200103A274B9A4234D882B20F239A4325
:1012E0004008083B184010432368D860002016E0EF
:1012F000012014E0082BDED0012010E0FFF768FE8B
:101300000028D8D100200AE0FFF73AFDF8E70120D5
:1013100005E0082B02D18020000285E7012001238F
:101320006A22A352023AA35200236367A36710BD47
:10133000FFF74EFE002800D076E70020EFE7FFF72A
:101340001FFDF7E70120EAE70120E8E7F369FFCF97
:10135000FFCFFFFFFFF4FF110038014000440040C1
:1013600000480040004C0040001002400024F400FF
:10137000D0190008EFFF0000836ADB0706D502687A
:1013800053682C490B40C16A0B435360836A9B0727
:1013900006D50268536828490B40016B0B43536024
:1013A000836A5B0706D50268536824490B40416B8A
:1013B0000B435360836A1B0706D5026853682049B4
:1013C0000B40816B0B435360836ADB0606D50268D2
:1013D00093681C490B40C16B0B439360836A9B0667
:1013E00006D50268936818490B40016C0B43936063
:1013F000836A5B060BD50268536814490B40416C45
:101400000B43536080235B03426C9A420AD0836A89
:101410001B0606D5026853680D490B40C16C0B438F
:1014200053607047026853680A490B40816C0B4354
:101430005360ECE7FFFFFDFFFFFFFEFFFFFFFBFF39
:10144000FF7FFFFFFFEFFFFFFFDFFFFFFFFFEFFF6C
:10145000FFFFF7FFFFFF9FFFF8B5CE46474680B579
:1014600006000D0017009946089B98463368DC6912
:101470002C40641B63425C41BC4257D1434601335C
:10148000F4D0FFF7E1F84B46C01A40452ED843464A
:10149000002B2BD033681A685207E7D5DA6912059A
:1014A000E4D5802212011A62EFF31080012282F348
:1014B000108831680B68204C23400B6080F3108843
:1014C000EFF3108082F3108831688B6893438B6050
:1014D00080F3108820238732B3500432B350043293
:1014E000B35064330022F254032020E0EFF3108065
:1014F000012282F3108831680B680F4C23400B6087
:1015000080F31088EFF3108082F3108831688B68C5
:1015100093438B6080F3108820238732B3500432CA
:10152000B35064330022F254032000E00020C0BC1A
:10153000B946B046F8BDC0465FFEFFFFF0B5C646EF
:1015400000B584B004000E0015001F008C23C358A2
:10155000202B00D086E0002900D188E0002A00D1AD
:1015600087E080235B0182689A4205D10369002BE2
:1015700002D1CB0700D57EE000239022A350043A8D
:101580002221A150E366FFF75FF880465C23E55215
:101590000233E552A36880225201934208D0002B07
:1015A00015D12269002A0ED16032FF21A15215E027
:1015B0002269002A03D160323149A1520EE0602233
:1015C000FF21A1520AE060227F21A15206E0802281
:1015D000520593420BD060220021A1526022A25AF0
:1015E00003928022520193420CD000251DE0226913
:1015F000002A03D160327F21A152EFE760223F2110
:10160000A152EBE72369002B01D000250DE0350046
:1016100000260AE023685B6A039A13402B80023598
:101620005E23E25A013A92B2E2525E23E35A9BB23F
:10163000002B12D000974346002220212000FFF704
:101640000BFF002819D1002EE4D023685B6A6A469C
:10165000127B134033700136E2E78C332022E250D4
:10166000002000E0022004B080BCB846F0BD01209C
:10167000F9E70120F7E70120F5E70320F3E7C0468B
:10168000FF01000030B583B0040090230022C25057
:10169000FEF7DAFF050022681268130710D42368EA
:1016A0001B685B0719D420238822A3500432A3505F
:1016B0000023E3662367083AA354002003B030BD3B
:1016C00080210C4B00930300002289032000FFF7C8
:1016D000C3FE0028E3D00320F0E78021054B0093F0
:1016E0002B000022C9032000FFF7B6FE0028DAD045
:1016F0000320E3E7FFFFFF0110B5041E30D088236D
:10170000C358002B22D088232422E2502268136879
:1017100001218B4313602000FFF736FD012814D010
:10172000A36A002B18D1226853680E490B405360FE
:10173000226893682A218B439360226813682939B1
:101740000B4313602000FFF79DFF10BD8433002280
:10175000C254FEF7C9FED6E72000FFF70DFEE2E710
:101760000120F2E7FFB7FFFF70B50C4D0C4E761B62
:10177000B61005D0002408CD01349847A642FAD10E
:1017800000F0EAF8074D084E761BB61005D000248D
:1017900008CD01349847A642FAD170BDEC19000873
:1017A000EC190008EC190008F4190008F0B5050060
:1017B000830749D0541E002A45D003000326CAB22D
:1017C00002E00135013C3ED301332A703342F8D1A7
:1017D000032C30D9FF220A40150215432A04154371
:1017E0000F2C34D92700103F3F093E01B4461E009C
:1017F0001A0010366644156055609560D560103249
:10180000B242F8D101373F01DB190F270C222740E4
:1018100022403C00002A0ED03E1FB608B400A44669
:101820001A001C1D644420C2A242FCD103240136CC
:10183000B6009B193C40002C05D0C9B21C19197088
:1018400001339C42FBD1F0BD03001400C0E7270028
:10185000E2E7C046034B10B5002B02D0024800F06F
:1018600005F810BD000000007D18000810B501004B
:1018700000230022002000F019F810BD70B5074DBC
:10188000074C641BA41005D0013CA300EB589847FB
:10189000002CF9D100F066F870BDC046F4190008BC
:1018A000F81900087047C0467047C046F0B5D646E4
:1018B0004F464646C0B5264F82B00600386892466D
:1018C00098468946FFF7EEFF224B1B680193A4233D
:1018D000019A5B00D558002D2ED06C681F2C30DC8F
:1018E000002E0FD1631C6B604B460234A400386895
:1018F0006351FFF7D9FF002002B0E0BCBA46B14601
:10190000A846F0BD882251462800A300EB18995044
:10191000873AA2408930FF30016811430160842179
:10192000404649005850022EDCD12B008D33FF3346
:1019300019680A431A60D5E715004D35FF35D550B3
:10194000CBE73868FFF7B0FF01204042D4E7C0463C
:1019500038040020E8190008F8B5C046F8BC08BCF7
:101960009E467047F8B5C046F8BC08BC9E46704716
:101970000000000000000000000000000000000067
:101980000000000000000000000000000000000057
:10199000010000000200000003000000040000003D
:1019A0000600000007000000080000000900000019
:1019B0000000000000000000000000000000000027
:1019C000010000000200000003000000040000000D
:1019D000010002000400060008000A000C001000CC
:0C19E000200040008000000110000020EA
:0819EC0055180008E90000088D
:0419F400C100000826
:1019F8000024F400010000000400000000000000C2
:101A080000000000FC02002064030020CC0300203A
:101A180000000000000000000000000000000000BE
:101A280000000000000000000000000000000000AE
:101A3800000000000000000000000000000000009E
:101A4800000000000000000000000000000000008E
:101A5800000000000000000000000000000000007E
:101A6800000000000000000000000000000000006E
:101A7800000000000000000000000000000000005E
:101A8800000000000000000000000000000000004E
:101A9800000000000000000000000000000000003E
:101AA800000000000000000001000000000000002D
:101AB8000E33CDAB34126DE6ECDE05000B000000F2
:101AC800000000000000000000000000000000000E
:101AD80000000000000000000000000000000000FE
:101AE80000000000000000000000000000000000EE
:101AF80000000000000000000000000000000000DE
:0C1E280000000000000000008005002009
:040000050800055D8D
:00000001FF
